:020000040100F9
:1000000038080020E5000001ED000001EF000001CC
:1000100000000000000000000000000000000000E0
:10002000000000000000000000000000F1000001DE
:100030000000000000000000F3000001F5000001D6
:10004000F7000001F7000001F7000001F7000001D0
:10005000F7000001F7000001F7000001F7000001C0
:10006000F7000001F7000001F7000001F7000001B0
:10007000F7000001F7000001F7000001F7000001A0
:10008000F7000001F7000001F7000001F700000190
:10009000F7000001F7000001F7000001F700000180
:1000A000F7000001F7000001F7000001F700000170
:1000B000F7000001F7000001F7000001F700000160
:1000C0000348854600F056F800480047B105000196
:1000D0003808002040BA7047C0BA70470138FDD1D7
:1000E000704700000448804704480047FEE7FEE7E9
:1000F000FEE7FEE7FEE7FEE795030001C100000111
:1001000030B50B46014600202022012409E00D46AF
:10011000D5409D4205D31D469540491B2546954037
:1001200040191546521E002DF1DC30BD03460B432D
:100130009B0703D009E008C9121F08C0042AFAD29D
:1001400003E00B780370401C491C521EF9D2704723
:10015000D2B201E00270401C491EFBD2704700225F
:10016000F6E710B513460A4604461946FFF7F0FFB6
:10017000204610BD064C0125064E05E0E36807CC7D
:100180002B430C3C98471034B442F7D3FFF79CFF45
:100190007C0800018C080001F7B5D4B004460E4677
:1001A00000205390052052900025002700BFEFF358
:1001B00010800090FF21453101A8FFF7D0FF00F02B
:1001C0004FFA05462448854218D101200003844295
:1001D00002D1002053902AE001204003844202D142
:1001E0004011539023E003200003844203D10120F7
:1001F000400253901BE0529857B0F0BD174885421B
:1002000013D101200003844201D153900FE001205B
:100210004003844201D1539009E00320000384424B
:1002200001D1539003E05298E6E75298E4E705AF16
:100230000137FF2241320A4901A8FFF777FF012069
:1002400000F04FF93146569A5398B84752900098AB
:1002500000F047F95298CFE7C440130085601300BF
:10026000A4060001F1B58AB0002009907D20C000ED
:1002700008900125AD020027002007907F200690FE
:1002800040240026002005900390200102900020C9
:1002900001903E490A98884206D83D4800686102AC
:1002A00088433B49086006E0394800680121C903DA
:1002B0000843374908607D21C9000A98FFF720FFED
:1002C0007D21C9000090FFF71BFF450100BF3048AA
:1002D00000687F21090288430190200201990843A8
:1002E0002B4908600520FFF7F9FE10E00120FFF719
:1002F000F5FE2748406B02210840002800D007E0A7
:100300000598411C05910899884200D900E0EDE765
:1003100000BF1F48C06B86B2AE4201D9771B00E018
:10032000AF1B0298874203D2E0B20390B8B20290AA
:10033000AE4201D3069400E007940699079840184E
:10034000C005000E04900498A04200D103E0049C74
:1003500009988742BBD800BF0D4800687F21090279
:1003600088430190039800020199084308490860F6
:100370000846406840084000486000BF04484068A4
:10038000042108400028F9D10BB0F0BD0090D00343
:100390000010024010B53E48C0690121090708431A
:1003A0003B49C861812000063A4908633A484861E0
:1003B0003A4808623A48006803218903884338496B
:1003C00008603421374800F073F836480069401C53
:1003D000002803D033480069002817D12C48406812
:1003E0000121090408432A4948600846406807215A
:1003F00009028843264948600846406809150843B1
:10040000234948602848FFF72DFF3FE021488069D5
:100410004409640123480078C006C00E04431D4807
:1004200084611B4800680121C9038843184908609A
:10043000084600687F21090288430446194800697C
:10044000000220431249086008464068012109045F
:1004500008430F494860084640680721090288435D
:100460000B49486008464068091508430849486038
:100470000846006A0D490840054908620846006AB6
:100480000849C968090208430149086210BD000013
:1004900000100240007000400F0800001800020029
:1004A00000100140000000200090D003FF00F8FF82
:1004B00070B504460D462A46214601200003FFF789
:1004C0006BFE70BD02E008C8121F08C1002AFAD1F5
:1004D00070477047002001E001C1121F002AFBD1C4
:1004E000704780F31088704770B504460D46206849
:1004F000002804D00721C9032068884201D90020C0
:1005000070BD2846216800F01FF86168884201D15B
:100510000120F5E70020F3E710B501460B684868B5
:1005200042085200180C000401246407A04208D1BC
:100530008A4206D30720C0030818824201D2012054
:1005400010BD0020FCE7000030B502460B4600213C
:10055000C94312E01078521C414000240BE04808C7
:10056000CD07ED0F002D01D0074D00E000256840BC
:100570000146601CC4B2082CF1DB18465B1E002843
:10058000E8D1C84330BD00002083B8ED044672B600
:100590000120C007204305490863206880F30888CC
:1005A00000BF6068804700BFFEE7000000700040A9
:1005B000284C002528492068884234D12021204633
:1005C000FFF7C2FF216A88422DD16068012808D157
:1005D000224920460830FFF787FF002801D01F4D31
:1005E00030E0606802280AD1412189042046143095
:1005F000FFF77AFF002802D04125AD0422E0174919
:1006000020460830FFF770FF002801D0134D19E095
:100610004121890420461430FFF766FF002811D0DD
:100620004125AD040EE00D48FFF776FF002801D00C
:100630000A4D07E041208004FFF76EFF002801D03B
:100640004125AD04002D02D02846FFF79FFF00BFD3
:10065000FEE700000040000111C011CA0080000147
:1006600070B5D2B00024002500BFEFF3108006461D
:10067000FF21453101A8FFF772FD01AC013498223A
:10068000074901A8FFF752FD0120FFF72AFFA04705
:1006900005463046FFF725FF284652B070BD0000E2
:1006A000E407000140BA7047C0BA70470138FDD175
:1006B00070470000F7B50325AD06286A82B01646DC
:1006C0000C46400840002862286A0221084328623C
:1006D000286A8007FCD46620686001272F61A86A19
:1006E000C005FCD5992068602F61A86AC005FCD5BB
:1006F000FF209130FFF7DAFFFF230133AB6268463A
:10070000EF60352169602F61A96AC905FCD5AB622C
:10071000A969EF60C9B205226A602F61AA6AD20591
:10072000FCD5AB62AA690902D2B211430180C807A5
:1007300002D0032005B0F0BDAB626869FF2108312B
:10074000884368616869C91E0843686102980002AD
:10075000483068600820A860EE602F61A86AC00574
:10076000FCD5FF200130A8620023F61CB0080ED093
:10077000B2081148006899006054060A09194E70C1
:10078000060C000E8E705B1CC8709A42F1D8FF20D8
:100790000130A8626869FF2108318843686168698F
:1007A00038436861286A800880002862286A3843D4
:1007B0002862002005B0F0BD8000000C03208006F8
:1007C0004169FF22083291434161426901210A4394
:1007D0004261026A920892000262026A0A4302625D
:1007E00070470000002003218906096A4908490072
:1007F0000322920611621146096A02221143032262
:100800009206116200BF03218906096A0222114083
:100810000229F8D0D1010322920691620321D1600E
:100820009F2151600121116100BF03218906896A5E
:10083000FF22013211409142F7D1032292069162C8
:10084000114688694969FF220832914303229206C2
:1008500051611146496901221143032292065161F7
:100860001146096A8908890011621146096A012244
:100870001143032292061162704700008C080001A8
:0C0880000000002038080000D404000133
:04000005010000C135
:00000001FF
